:020000020000FC
:1000000009C008C007C006C005C004C003C03FC087
:1000100001C000C0F8940FEF0DBF02E00EBF02D088
:100020007894FFCF0FEF0AB90FEF07B90FEF04B9BC
:1000300020E030E040E0EE24FF24BB24CC24332435
:10004000442402E0502E0FE7502F00E0009381007F
:100050000FE700938A0000E000938B0000E000931C
:100060006F0001E30093800009E00093810000E04D
:100070000093B10002E00093700009EF0093B30019
:1000800002E00093B00001E00093B10008950F93E7
:100090000FB70F93339509F44395203011F41FD017
:1000A00009C0213011F44CD005C0223011F479D0B0
:1000B00001C0A8D000E430170CE9400761F430E03B
:1000C00040E0EE24FF24BB24CC2433244424239595
:1000D000243009F420E00F910FBF0F91189533944D
:1000E00009F4439406ED039DE02CF12C06ED049DEC
:1000F000F00C00E0039DF00C0E2D059DB02CC12CE2
:100100000F2D059DC00CE6E6F2E0EC0D08F4F3952A
:1001100004910503A12CFA0CE8E6F3E0EF0D08F4D6
:10012000F395D49000E000938B00D0928A0001E315
:10013000301601E0400619F400E0302E402E0895FC
:10014000339409F443940FE0039DE02CF12C0FE06D
:10015000049DF00C01E0039DF00C0E2D059DB02CCC
:10016000C12C0F2D059DC00CE6E6F2E0EC0D08F465
:10017000F39504910503A12CFA0CE8E6F3E0EF0DEA
:1001800008F4F395D49000E000938B00D0928A009D
:1001900001EF301600E0400619F400E0302E402E4A
:1001A0000895339409F4439401E4039DE02CF12C69
:1001B00001E4049DF00C01E0039DF00C0E2D059D63
:1001C000B02CC12C0F2D059DC00CE6E6F2E0EC0D25
:1001D00008F4F39504910503A12CFA0CE8E6F3E08A
:1001E000EF0D08F4F395D49000E000938B00D092CB
:1001F0008A000CEC301600E0400619F400E0302EC6
:10020000402E0895339409F443940CEA039DE02CA6
:10021000F12C0CEA049DF00C01E0039DF00C0E2D76
:10022000059DB02CC12C0F2D059DC00CE6E6F2E01B
:10023000EC0D08F4F39504910503A12CFA0CE8E603
:10024000F3E0EF0D08F4F395D49000E000938B00F9
:10025000D0928A0009E9301600E0400619F400E067
:10026000302E402E0895000306090C101316191C99
:100270001F2225282B2E313336393C3F4144474934
:100280004C4E515355585A5C5E60626466686A6BA6
:100290006D6F70717374757678797A7A7B7C7D7DF9
:1002A0007E7E7E7F7F7F7F7F7F7F7E7E7E7D7D7C6B
:1002B0007B7A7A79787675747371706F6D6B6A6812
:1002C000666462605E5C5A585553514E4C494744CF
:1002D000413F3C393633312E2B2825221F1C19165D
:1002E00013100C09060300FDFAF7F4F0EDEAE7E459
:1002F000E1DEDBD8D5D2CFCDCAC7C4C1BFBCB9B748
:10030000B4B2AFADABA8A6A4A2A09E9C9A989695B5
:100310009391908F8D8C8B8A888786868584838342
:1003200082828281818181818181828282838384B0
:1003300085868687888A8B8C8D8F909193959698E9
:100340009A9C9EA0A2A4A6A8ABADAFB2B4B7B9BC0C
:10035000BFC1C4C7CACDCFD2D5D8DBDEE1E4E7EA5E
:10036000EDF0F4F7FAFD0003808386898C90939674
:10037000999C9FA2A5A8ABAEB1B3B6B9BCBFC1C48E
:10038000C7C9CCCED1D3D5D8DADCDEE0E2E4E6E8EA
:10039000EAEBEDEFF0F1F3F4F5F6F8F9FAFAFBFC1D
:1003A000FDFDFEFEFEFFFFFFFFFFFFFFFEFEFEFD69
:1003B000FDFCFBFAFAF9F8F6F5F4F3F1F0EFEDEBEA
:1003C000EAE8E6E4E2E0DEDCDAD8D5D3D1CECCC987
:1003D000C7C4C1BFBCB9B6B3B1AEABA8A5A29F9C00
:1003E000999693908C898683807D7A7774706D6AF4
:1003F0006764615E5B5855524F4D4A4744413F3CEC
:10040000393734322F2D2B28262422201E1C1A186F
:1004100016151311100F0D0C0B0A0807060605041C
:1004200003030202020101010101010102020203B0
:10043000030405060607080A0B0C0D0F101113150F
:1004400016181A1C1E20222426282B2D2F32343752
:10045000393C3F4144474A4D4F5255585B5E6164B9
:0A046000676A6D7074777A7D8083FF
:00000001FF
